:1093400020496E697469616C697A696E67202000D2
:109350003232336520496E70757420506F727420FC
:099360000033302E3120202000E2
:1065F700C105C108C101C104C1064114DA00421432
:10660700D70000C187C18043149C01141643149F0F
:106617000114164414A3FFFFFFFFC1034114D9005F
:04662700411496FF85
:1069F000EFFD3395E0FC74A32DF58274143CF58310
:106A000022901300124D5989828A832290093DE019
:106A1000D36480F8EE64809822EEFD3395E0FC7438
:106A2000982DF58274143CF58322FE75F02DEF123B
:106A30004D44E5822EF582E43583F5837401F090B0
:106A40001600E004F02274002FF582E43406F5838A
:106A50002290161B124D7990000512493EFF9000BE
:106A60000612493EFD90000402493E901600E025C2
:106A7000E02416F582E43405F583227B017A167949
:106A80000890161B124D7990000312493EFF901496
:106A9000D6E06F22901600E0FF24DEF582E4340594
:106AA000F58322EDFF3395E0FEEF25E0FFEE33FEA8
:106AB00022FBEAC4F854F0C8EBC4540F48901749BD
:106AC000F022E475F001024A5E129262EE547FFFFA
:106AD00022901600E0FFC32274FB2FF582E43413EA
:106AE000F583223EF583EAF0A3EBF0223EF583E046
:106AF000FAA3E022EC25E02426F8E6FA08E6229044
:106B000014D77427F0A37410F02290149C024D59EE
:106B10007B017A147916024D7990149F024D591217
:056B20004D59024DD4A7
:109A370075840F75A4357580C075A57C75A7FF75EE
:069A4700E11775E3442263
:0F9ADA00E4F584759A4075F809759D04C2FA2267
:104FE400E4F584758850758921F58EF58D75C908A9
:104FF40075CDFF75CCC075CBFF75CAE075C804F5D7
:02500400842204
:109A6200E4F584759105759852758401759810F521
:029A720084224C
:108AD100E4FFFE75840F438A0353A1DFF58475B764
:108AE1003075840F43A120438901758D01758F0174
:108AF100758E040FBF00010EEF640F4E70F54389B0
:108B010002E58920E4130FBF00010EBE0FF3BFFF82
:0C8B1100F0E4F58443EF1080E875970253
:018B1D002235
:0D9B420075A89275B81075E60875E7402209
:109A7400E4F58475D84075D98375DA3175DB31D254
:029A8400DE22E0
:109A4D00129A37128AD1124FE4129A74129A621234
:059A5D009ADA029B42B1
:0A9BC6007F021299DB7F040299DB95
:02762100AC07B4
:10762300E490174AF0ED4430901748F0E4FDEDFF85
:107633003395E0FE74FC2FF58274053EF583E06C10
:10764300705890174A04F0ED126AA574952FF582CD
:107653007402126AEC126AB1EB540FF9126AA37442
:10766300D92FF5827401126AECFB74952FF582749D
:1076730002126AE374F02FF5827400126AECFB7451
:10768300D92FF5827401126AE3126AF4FB126AA31A
:1076930074F02FF5827400126AE30DED6404708EAA
:1076A30090174AE0700C126AF4126AB1AF03EF54F8
:1076B3000FF9E9C454F0F9E59A20E7FBE4F59BE5FB
:1076C3009A20E7FB901748E0F59BE59A20E7FB90AB
:1076D3001749E0F59BE59A20E7FB899BE59A20E7AC
:0176E300FBAB
:0176E4002283
:0579AF0090175AEFF0F3
:1079B400124DAE79D30079E00179ED0279FA037AB8
:1079C40007047A14057A21067A2E0700007A397F93
:1079D4000612676F90175B7405F080597F06125F7B
:1079E4000D90175B7406F0804C7F06128030901760
:1079F4005B7407F0803F7F061273CA90175B7408AC
:107A0400F080327F0712676F90175B7409F080254E
:107A14007F07125F0D90175B740AF080187F0712BE
:107A2400803090175B740BF0800B7F071273CA9041
:107A3400175B740CF0D282C29590175BE0FF90172D
:0A7A44005AE0FD127621D295C282AD
:017A4E002215
:057A4F0090175CEFF050
:107A5400124DAE7A73007A80017A8D027A9A037A93
:107A6400A7047AB4057AC1067ACE0700007AD97FD2
:107A74000812676F90175D740DF080597F08125FCC
:107A84000D90175D7412F0804C7F081280309017AF
:107A94005D740FF0803F7F081273CA90175D7410F5
:107AA400F080327F0912676F90175D7411F08025A2
:107AB4007F09125F0D90175D740EF080187F091214
:107AC400803090175D7413F0800B7F091273CA9095
:107AD400175D7414F0D282C29690175DE0FF901780
:0A7AE4005CE0FD127621D296C2820A
:017AEE002275
:058A280090175EEFF065
:108A2D0024FA601704702B90175F741DF090164494
:108A3D007403F07B277D2A7F1D801290175F741CB5
:108A4D00F09016447402F07B117D1F7F1C1270D1C3
:108A5D00800A90175EE0FFA3F0125C92D282C2945E
:108A6D0090175FE0FF90175EE0FD127621D294C261
:018A7D008276
:018A7E0022D5
:05897800901760EFF014
:10897D0024FA601704702A901761741BF090164446
:10898D007401F07B287D2B7F1B8011901761741A69
:10899D00F0E4901644F07B127D207F1A1270D18086
:1089AD000C901760E02415FFA3F0127CC0D282C298
:1089BD0097901761E0FF901760E0FD127621D29736
:0289CD00C28264
:0189CF002285
:0F9AE9009014157407F0D294D295D296D297228A
:10926200C2AC126B0AEF12498D90149D126AC2129F
:109272006B0A74019014966B7008E965827003EAB8
:0D9282006583700690149C126B10D2AC2214
:108C5000126B19C003C002C001126B0AD082D0830C
:108C6000D0E06B7008E965827003EA6583602B12BF
:108C70006B19124925FF1298789014A0126AC2123B
:108C80006B1974019014966B7008E965827003EAA1
:0B8C90006583700690149F126B102289
:1072E10090177CE584F0ACA89012E5124D59E94A5B
:1072F10070030273C953A87DE4F58453F87F901499
:10730100DCF0A3F0C2B39013D3E0FFB401189012E4
:10731100CCE0C313FE7402A806088002C333D8FC74
:107321009014DCF08059EFB402169013A4E0FF74BE
:1073310001A807088002C333D8FC9014DDF0803F18
:107341009013D3E0B403389012D3E0C31314601543
:1073510014601A14601F146024240470229014DD38
:107361007410F0801A9014DD7420F080129014DDF6
:107371007440F0800A9014DD7480F08002D2B33042
:1073810002079014DCE04440F0C2FAE4FF0FEFB4CE
:1073910032FB53F87FE59A20E7FB9014DCE0F59B84
:1073A100E4FF0FEFB432FB53F87FE59A20E7FB903F
:1073B10014DDE0F59BE4FF0FEFB432FBD2FA901736
:0873C1007CE0F584AF048FA805
:0173C90022A1
:035006000277A48A
:1077A400C0E0C0F0C083C082C0D075D000C000C0AB
:0D77B40001C002C003C004C005C006C0072C
:1077C100C39014D8E094F89014D7E0942A5003128F
:1077D1006AC2901415E014F0E0C3940750067426B1
:1077E100F0128C50901415E0FF131313541FFEEF89
:1077F100540790177DF0AF06EF24FE601814601F48
:107801001460262403702E90177DE0FF6407602525
:10781100128A28802090177DE0FF1279AF801690A0
:10782100177DE0FF127A4F800C90177DE0FF64070F
:0B7831006003128978758AFF758CFFD8
:10783C00D007D006D005D004D003D002D001D000A0
:0B784C00D0D0D082D083D0F0D0E0324A
:109ACA0075F002EF900580124D44ECF0A3EDF02200
:0A9BD000AE077F8B126AC902926291
:0A9BDA00AE077F82126AC902926290
:0A9BE400AE077F83126AC902926285
:10845100E4FE126A0C5012EE1269F1E0F46007EECC
:10846100126A1BE004F00E80E99014A7E0FE126985
:10847100F1EFF0126A19E4F0FE126A0C5012EE12DA
:1084810069F1E0B4FF079014A7EEF0803B0E80E99C
:10849100E49014A7F0901498E0FD7E01126A0C504C
:1084A10027EEFB3395E0FA74982BF58274143AF5B4
:1084B10083E0FCD3ED6480F8EC6480984007AD0460
:0B84C1009014A7EEF00E80D4129BDA9E
:0184CC00228D
:0576E500901762EFF0B8
:1076EA00E4FF90093DE0D36480F8EF648098506B22
:1076FA001269F0E0FE901762E0FDEE6D70591269B2
:10770A00F074FFF0126A1F74FFF0901763747FF031
:10771A00E4FE126A0C501CEE6F6015126A19E0FD45
:10772A00901763E0C36480F8ED6480985002EDF02E
:10773A000E80DFE4FE126A0C5021EE6F6016126AA8
:10774A0019C083C082E0FD901763E0FCC3ED9CD0B2
:10775A0082D083F00E80DE0F0276ECE49014A7F05C
:10776A00FF90093DE0FED36480F8EF6480985010E2
:10777A001269F0E0F4601A9014A7E004F00F80E1B7
:10778A00EE14FF9014A7E0FED3EF126A114002EF45
:09779A00F0901762E0FF129BE47D
:0177A30022C3
:109878007584014398028F99E59870047F018002EE
:0A9888007F00EF20E1F2E4F58422F6
:1099DB00E4F5844398028F99E59870047F01800227
:0799EB007F00EF20E1F222F2
:10928F00E4FEC3EF126A115023E4FDC3EF6480F8CC
:10929F00ED6480985013E4FCC3EF6480F8EC6480B5
:0C92AF009850030C80F20D80E20E80D677
:0192BB002290
:109A8600AE07ED60047F8F80027F8E126AC9029254
:019A9600626D
:10409A00E490093DF0FBFAF99012E5124D7975FFAB
:1040AA00DE75FFADE4F5E6F5E7129A4D129AE912CC
:1040BA00962F129AA87BFF7A9379509016F8124D90
:1040CA00797A9379401290881298E0E4F58475D44D
:1040DA008475D48475D10375D340D281128E01D2EE
:1040EA00AFD2FFE4901600F09014D6745AF0FF1283
:1040FA009B4F43F602E49014A7F0901600F0900943
:10410A003DE0FF3395E0FE901600E0D39FEE648019
:10411A00F8748098501FE0FF24A3F582E43414F564
:10412A008374FFF074982FF582E43414F58374FFD6
:10413A00126A3E80C9E41248241286A91296B41261
:10414A009BEE1272E17F391299DBC2011298FAEFE3
:10415A00640160030244F8129539EF64B060030207
:10416A0044F8901607F0901600F0126AD1942D5078
:10417A001074A92FF582E43414F583E4126A3E80A0
:10418A00E9E4901600F0126AD1941B501AE0FE245A
:10419A0000126A49E0FD74DE2E126A9BEDF0126A83
:1041AA0046E4126A3E80DFC21C1298FAEF60FA12E5
:1041BA009539901601EFF05480FFE4FCFDFEEF7094
:1041CA0003024336E0FF64C07003024336EF64B073
:1041DA007003024336901607E004F0901601E0548B
:1041EA007FFF901603F07419D39F500DE0FF9426B9
:1041FA005007EF24F2A3F0802A901603E0FFE4D3DD
:10420A009F500AEF94185005A3EFF08016EFB429D7
:10421A00089016047419F0800AEFB42C069016045C
:10422A00741AF0901604E0FFC3941B5029126A46D0
:10423A007401F09014D9EFF09014A8E0FF901604DE
:10424A00E06F600A9013D3E0B40603126D7A9016F9
:10425A0004E09014A8F0E4901605F0A3F01298FA7E
:10426A00EF60FA129539901602EFF01298FAEF60A1
:10427A00FA129539AD07901602E0FF901605E0F0A4
:10428A00A3E04FF0901605E0FEA3E07806C333CE14
:10429A0033CED8F9F0EE901605F0AF05E0F0A3E0C2
:1042AA004FF0901603E075F002900580124D44E03D
:1042BA00FEA3E04E702F901600F0126AD1940550BA
:1042CA000C901603E09000F8126A2A80EDE490162A
:1042DA0000F0126AD19404500C901603E09001E1A8
:1042EA00126A2A80ED901603E0FF901605E0FCA3FF
:1042FA00E0FD129ACA901603E0FF24A9F582E4347D
:10430A0014F5837401F09014A2EFF0C39419400CD1
:10431A00E0FFD394265005EF24F280049014A2E023
:10432A00901497F0201C05129204D21C901601E0FA
:10433A0064C060030241B39013A3E0601E9013D3DC
:10434A00E0B4020812891B300502C2059013D3E0BB
:10435A00B40608128D2E300802C208E4901600F046
:10436A00126AD1941B40030244F874DE2F126A9B2E
:10437A00E060030244AC901600E02400126A49E0AF
:07438A00640160030244AC72
:10439100901621F0A3F0901621E0FEA3E0FFC39454
:1043A10004EE64809480504590074975F07DEF12CA
:1043B1004D44EE75F07DA42583F583C083C08290C2
:1043C1001600E0FFD082D08375F005124D44E05411
:1043D1000F6012901621E0FCA3E024DAF582740547
:1043E1003CF583EFF0901621126AC280A99013A3C5
:1043F100E07008901600E0FF128451901600E0FF73
:10440100126A6F7414F0A3E4F0EF25E02496F582AC
:10441100E43400F583C083C082E04410FFA3E0D000
:1044210082D083CFF0A3EFF09013A3E07003024496
:10443100F2D205D2089013D3E0FF6402703F9012CC
:10444100E2124D59901600E0FE75F005A4F5828543
:10445100F08312493E540F70047D0180027D00ED0E
:10446100540FFD9012E2124D5975F005EEA429F991
:10447100EA35F0FA12492554F04D12498DEF6406E0
:104481007020901600E0FF24FB126ADBE070047ECE
:104491000180027E00126AD8EEF0126AD8E0FD12A5
:0844A1009A8612501B129BEEDB
:1044A9000244F2126A94E0B4010B126A46E0700504
:1044B9001276E58034126A94E06401702C126A461F
:1044C900E064017024126A6BE0FCA3E0D39400EC71
:1044D9009402400EEF126A6F74FE75F000124A5E84
:1044E9008007126A6BE4F0A3F0126A3F02436A1272
:0A44F9009914EF640160030245DF2F
:1045030012955D901621EFF030E738E0901496F0A5
:10451300246824FC501D24E1601324D26003024567
:10452300DF126AFF9012D0126B1F0245DF129A202E
:104533000245DF901496E02468901414F05403F0BD
:104543000245DF901496E0124DAE45CD8C45D78DD4
:10455300456F9045779245879345B19445BB954503
:10456300C39645979745A79D000045DF12481874E9
:1045730092F08068901621E0FF129BF790149674D6
:1045830093F08058901621E0FF128DBC901496741E
:10459300F0F08048901621E0FF129B5C9014967413
:1045A3009DF08038901621E0FF129581802E9016A1
:1045B30021E0FF129B0780241248187496F0801C98
:1045C300901621E0FF129B8D8012901621E0FF12BE
:0C45D3009B168008901621E0FF129B252B
:0945DF001297EBEF70030246ACE9
:1045E80012916B901621EFF0124DAE465B014656C4
:1045F80002466E04462205461B0646300746290831
:10460800463E0946370A464C0B46450C46630D00A4
:1046180000469D126A017FFF802F126A017F018088
:1046280028126A017FFE8021126A017F02801A1215
:104638006A017FFD8013126A017F03800C126A01F0
:104648007FFC8005126A017F04124DD880131297EF
:10465800CD800E901306126B1F8006901303126B09
:104668001F1272E1802F300312B2023002047F89D8
:1046780080027F8A901603EFF0800FE49006CFF057
:104688001299ABC2027FBA1292621272E1901603BB
:05469800E0FF1298781C
:10469D001297EBEF60030245E8126AFF129BEE30B2
:1046AD0004109014D6E0FF7BFF7A9379611289D0C4
:1046BD00C20430060A9014D6E0FF129947C2067B59
:1046CD00017A1679081295EBEF700302415490169A
:1046DD000AE0124DAE474304475405470D144701F8
:1046ED001647051747121A472C1B47371D473D1E06
:1046FD0000004771D2028002C2021272E1024771BC
:10470D00D2030247717B017A167908901618124D63
:10471D0079124925FE9014D6E0FF6E704780059002
:10472D0014D6E0FF1299F2024771129C10024771E4
:10473D00129C56024771126A7B702930021E126A52
:10474D0051FB1285C08015126A7B701830020D1254
:10475D006A51FB128143129514129BEE9014D6E010
:10476D00FF1299602002030246CC90160AE01460F5
:10477D001A24FA602114604C240660030246CC1200
:10478D0047EB9006CFF01299AB80331247EB1248EE
:10479D0024129BEE8028124801126A65FD900005D7
:1047AD0012493EFBC00390161E124D599000061281
:1047BD00493E901670F0D003127DF0129BEE129BC5
:1047CD00A50246CC124801126A65FD9000051249FA
:0E47DD003EFB126EA0129BEE129BA50246CC74
:1047EB00129A977B017A167908901618124D7990C8
:1047FB00000312493E22129A977B017A1679089090
:10480B00161E124D7990000312493EFF229016217D
:10481B00E0FF129C68901496229006CFF01295142C
:04482B00129BC622F4
:1094A500E0FEA3E0A60608F6E4F584C2AF43B701E3
:1094B50022E475F001124A7485F082F58322EEF0FC
:0594C500A3EFF0A3225B
:10913400AB84A2AF921DE4FCFDED90171C124CF61B
:1091440090171E786C1294A5438F02438F0118E682
:10915400FE08E6F5828E83E4F053B7FEF58FA21D78
:0691640092AFAF038F84FF
:01916A0022E2
:028F5400AB056B
:108F5600AA84A2AF921EE4FCFDED901720124CF6F7
:108F6600EBFF3395E0FEEFF44E601C901722786E0F
:108F76001294A5758F0118E6FC08E6F5828C83EB42
:0F8F8600F053B7FEE4F58FA21E92AFAF028F84B7
:018F950022B9
:108A7F009016E31294C3ECF0A3EDF0A3EAF0A3EB8E
:108A8F00F09016E7E07002A3E060369016E3E0FE88
:108A9F00A3E0FFA3E0FCA3E0F5828C83E0FD128F3F
:108AAF00549016E774FFF5F0124A5E9016E5E475E0
:108ABF00F001124A5E9016E3E475F001124A5E80EF
:028ACF00C022C3
:089C0000E4900BB2F0A3F02286
:10945900900BB2E0FEA3E0FF129134900BB2E0FE54
:10946900A3E0FF7C0B7DB47B007A04128A7FE49031
:069479000BB2F0A3F0228B
:0A854900A9059016E9EEF0A3EFF08B
:10855300EE54FCFE900BB2E0FCA3E0FD7002EE6C67
:108563006042ED4C60031294599016E9E0FEEE541C
:10857300FCFE7F00900BB2F0A3EFF09016EB129489
:10858300C3740BF0A374B4F07E049016EB1294B68C
:10859300E493FD9016ED1294B6EDF0EF1F70011EFB
:1085A300EF4E70E69016E9E0FCA3E0FDEC5403FC0B
:0C85B30074B42DF582740B3CF583E9F0E4
:0185BF002299
:1090FC009016D51294C3124D799016DA74FFF5F0D0
:10910C00124A7445F060209016D5E475F001124AAD
:10911C0074AFF0FE9016D7E475F001124D6212494F
:08912C0025FD12854980D222C5
:10662B004215D60000421581000042157C0000C1C6
:05663B0014C113C1129F
:10904E0090157CE475F001024A5ED39015D7E0903E
:10905E0015D69400E06480948022E0FEA3E0248381
:10906E00F58274152290157CF0A3F02274FFF5F0B2
:0A907E00024A5EFCE5F064404C225B
:10947F00C213C214E49015D6F0A3F0901581F0A397
:10948F00F0A3F0129073901577F0A37440F0E4906E
:06949F00157FF0A3F0228E
:10992E00E4F5848FC343C30175C04475CF8EC2C3A3
:09993E0043E60290157E04F022BC
:109A9700E4F58420C7FDC2C212947FE490157EF0DE
:019AA700229C
:0B9BA500E4F584D2C290157E04F0228B
:0D9B4F00AE0712992E90157BEFF002947F67
:1094CA00E4901764F0A3F0301302FF222014FDD2B7
:1094DA0013901579E4F0A37410F09015C4EFF0E43A
:0494EA00A3F07F016B
:0194EE00225B
:1092BC0030130A901579E07002A3E070037F00224E
:1092CC0090157912907A9015C5E0FE04F074C62EB4
:0C92DC00F582E43415F583EFF07F0122E9
:0B9BB000301307C213D214129AF822DF
:0E9AF800AF84E4F58420C7FDC2C4D2C58F84BC
:019B0600223C
:10871A009016DD124D7990157EE07002FF229016B8
:10872A00E0E0FE6005D3941040037F00221294CA51
:03873A00EF6049A4
:10873D00E49016E2F09016E0E0FF9016E2E0FEC342
:10874D009F501F9016DD124D598E82758300124970
:10875D003EFF1292BCEF7002FF229016E2E004F091
:10876D0080D3E4901580F0129BB09016E1E0700379
:09877D002014FD901580E0FF229C
:038786007FFF2250
:0B7AEF00901724124D79901727EDF03E
:107AFA0012905850037F002290157C1290683EF530
:107B0A0083E0FF12904E12908170031290739015C9
:107B1A0077129051E4FE901727E0FDEEC39D503591
:107B2A00EEC39F503090157CE0FC12906A3CF583BE
:107B3A00E0FD901724124D598E82758300ED12498B
:107B4A009F12904E129081700312907390157712C3
:107B5A0090510E80C1EEC39F501412904E12908124
:107B6A0070031290739015771290510E80E790155A
:107B7A00D612907A901727E0FEEFC39E5002800239
:027B8A00AF0644
:017B8C0022D6
:0C9B690012905840047F0180027F00220F
:035018000268B774
:1068B700C0E0C0F0C083C082C0D075D000C000C0A7
:0368C70006C00701
:1068CA00C21FAFC1EF124DAE69000869001069100E
:1068DA0018691520692228694F30695A3869616038
:1068EA00695C68696170695C7869688069689069DF
:1068FA00BCA0000069CA9015C4E0F5C2C2C59015D3
:10690A00C3E4F00269CC9015C5802890158074FD07
:10691A00F0D2C4D2C50269CC9015C5E0FF9015C368
:10692A00E0C39F5014E0FF04F074C62FF582E434EC
:10693A0015F583E0F5C20269CCD2C4901580E4F063
:10694A00C2140269CCD2C590158074FEF00269CCDB
:10695A008065D2120269CC901576E4F08064D390F7
:10696A001578E0901577129060403F12907A901552
:10697A0076E07006E5C2F0E004F0901581129068A6
:10698A003EF583E5C2F0901581129051FEE5F06460
:10699A00404E7006901581F0A3F0901576E014F041
:1069AA0070209015D6129052801890157F74FFF0BF
:1069BA00801030120DC2129015C3E4F0D2C58002C5
:1069CA00D21F301F0EC2C6D2C6C2C5C2C4D2C2C2EC
:0569DA001FC214C2C33E
:1069DF00D007D006D000D0D0D082D083D0F0D0E076
:0169EF003275
:05500900A2C7E433FF23
:01500E00227F
:109892007B01E49016F3F0227422F0A3EFF0A322EE
:0A98A2007B01E49016F3F07D042230
:0B8F96009016EF124D799016F2EDF0EE
:108FA100E49016F4F09016EF124D599016F2E090FD
:108FB10016E0F09016F3E09016E1F0E4FF12871A44
:108FC100EFB4FF0D9016F4E0FE04F0EEC3940340FD
:038FD100D47E004B
:018FD400227A
:0695EB0090174B124D79B0
:1095F1007E007F007D10124E0790174B124D597D52
:0B96010010127AEFEF7002FF227F01D1
:01960C00223B
:1089D00090168F12989A7413F0124925901692F0FF
:1089E00090000112493E901693F090000212493E09
:1089F000901694F090000312493E901695F0900066
:108A00000412493E901696F090000512493E9016C9
:108A100097F090000612493E901698F07A16798FDA
:088A20001298927D0A028F9664
:1099470090172812989A7403F0A374FFF07A177986
:09995700281298927D04028F96FB
:1099F20090172C12989A741CF0A374FFF07A1779BE
:079A02002C1298A2028F96BE
:10996000E4901730F0A3EFF0A3740AF0A3EFF07ABD
:099970001779301298A2028F96BB
:108F110074FFF5F0024A5E7403F0A374E8F0A3E570
:108F210084F0E4F58422D2C4D2C5D2C2C2C3E49093
:108F3100177FF0FF22EFF0A3ECF0A3EDF0A3024DB9
:108F410079E51C851DF0024A5EE025E044A0F5C2EA
:038F51007F032279
:06501200C2C253E6FD22BC
:0671DC00901661128F36CF
:1071E20090166A128F1820C7FDC2C4D2C2D2C5E45B
:1071F200FF90177FF030C3FDAEC1EE124DAE721C90
:1072020000721F08721F10722D18723720723F28E9
:10721200729230729A380000721C0272A2EF7006EB
:10722200901661128F4AC2C50272A8901662E0F5EA
:10723200C27F05807190177F7403F08069EFB405F7
:107242000B901662A3E0F5C27F06805AEF640670C7
:107252002D901669E0901664700875F001124D6267
:107262008003124D59124925F5C2901667128F11EB
:10727200901667E07002A3E0702C7F078028EFB4BD
:107282000706D2C47F09801E90177F7405F080160E
:1072920090177F7404F0800E90177F7406F08006BA
:1072A20090177F7401F0EFB40904C2C380279017CE
:1072B2007FE0B4030D90166A128F1145F06003123D
:1072C2008F2790177FE06008C2C5D2C4C2C3800571
:0E72D200C2C30271F720C7FD90166CE0F58470
:0172E000228B
:066C5000901679128F3648
:106C5600901681128F1820C7FDD2C2C2C4D2C5E4D5
:106C6600FF90177FF030C3FDAEC1EE124DAE6C99AA
:106C7600006C9C086C9C106CC1186CCB206CD328E3
:106C86006CEE306CF6386CFE406D0E506D3558006B
:106C9600006C99026D3BC2C5EF7009901679128F90
:106CA6004A026D41EF64016003026D41901679E07E
:106CB60025E044A1F5C27F04026D4190167AE0F505
:106CC600C27F05807690177F7403F0806EEFB4055F
:106CD6000B90167AA3E0F5C27F06805FEFB4060636
:106CE600D2C57F018055801890177F7404F0804BC1
:106CF60090177F7406F08043EFB404047F02803B54
:106D060090177F7405F0803390167CE475F00112BD
:106D16004D62E5C212498D90167F128F1190167F33
:106D2600E07002A3E07004C2C280107F02800CD221
:106D3600C47F09800690177F7401F0EFB40904C27E
:106D4600C3802790177FE0B4030D901681128F1130
:106D560045F06003128F2790177FE06008C2C5D206
:106D6600C4C2C38005C2C3026C6B20C7FD901683E4
:036D7600E0F584C1
:016D790022F7
:106FBA009016A3EFF09016A6124D799016A4ECF055
:036FCA00A3EDF044
:106FCD00751E00543FF51F543F604BC37440951F11
:106FDD00FFE4951EFE9016A9E0FCA3E0FDC39FEC17
:106FED009E50068C1C8D1D80048E1C8F1D1270A84A
:106FFD0060037F02229016A4128F429016ABE070B0
:10700D00069016A7128F42C39016AAE0951DF09018
:10701D0016A9E0951CF09016A9E0F51CA3E0F51D4E
:10702D00D3E51D9400E51C9400406DE51D9440E5ED
:10703D001C9400500F1270A860037F0222E4F51C0F
:10704D00F51D80DC9016A3E0FFA3E0FCA3E0FDA3FB
:10705D00124D59901667E4F0A37440F09016ABE012
:10706D00901669F01271DC90177FE060037F0222A9
:10707D0074C0251DF51D74FF351CF51C9016A4E478
:10708D0075F040124A5E9016ABE070949016A7759D
:0A709D00F040124A5E02702D7F00E1
:1070A700229016A3E0FFA3E0FCA3E0FDA3124D5935
:1070B700901667E51CF0A3E51DF09016ABE090165F
:0A70C70069F01271DC90177FE022DF
:109A090090167FE4F0A304F0126C5090177FE06089
:079A1900037F01227F002200
:1098AC0090177EEBF07B017A17797E9016A9E4F085
:0A98BC00A304F0E4A3F0126FBA2237
:10960D00C0079016BBE0FFA3E090167FCFF0A3EF4D
:10961D00F0D007126C5090177FE060037F01227F1E
:02962D00002219
:1098C600C0079016C3E0FFA3E09016A9CFF0A3EF60
:0A98D600F0E4A3F0D007126FBA22ED
:10664000026314F6026514F6016907016707016B1E
:10665000000162005014E30001FF00FF000001018F
:106660000000FF00FF0100C1184214E100004114C6
:02667000E00048
:10923400901735024D59D3ED9408EC648094802244
:10924400D3ED9410EC6480948022C3ED94F8EC6424
:0E92540080947F22C3ED94F0EC6480947F221E
:0587F300901734EFF0C7
:1087F800E5642401FFE43563FAA9077B01A3124D60
:108808007912923474019015766B7008E96582705C
:1088180003EA6583700C7B017A1479F69017351298
:108828004D79129234EB8A8389826401700AE56675
:1088380065827004E56565836019901734E0856486
:1088480082856383F0129234AF018A638F64901734
:0388580034E0F019
:01885B0022FA
:10916B0053E6F7E564B56609E563B56504E4FF808E
:10917B00210566E566AE657002056514F5828E8382
:10918B00E0FF7476B5660B7415B5650675651475D9
:05919B0066F643E60842
:0191A00022AC
:1097EB0053E6F7E564B56609E563B56504E4FF8008
:0C97FB0008856682856583E0FF43E60870
:01980700223E
:03501E000263BE6C
:1063BE00C0E0C0F0C083C082C0D075D000C000C0A5
:1063CE0001C002C003C004C005C006C0079013D4AC
:1063DE00E060030265DC30DF02C2DFE5B05407F592
:1063EE006965676010E5696567F56B7568035569E2
:1063FE00F562856967E56860661568E5687060E551
:10640E0069540370069014E07403F0E56230E01AEC
:10641E009014E0E0FE70047F01800CEE54FE9014A8
:10642E00E0F030E1057F0D1287F3E56230E11A905E
:10643E0014E0E0FE70047F02800CEE54FD9014E038
:10644E00F030E0057F0D1287F3E56B30E211E56960
:10645E0020E20C9014E17401F0A374F4F0D2183021
:10646E0018269014E174FFF5F0124A5E9014E1E0E4
:10647E007002A3E07006C218D204800CE5B030E2C0
:0E648E0007C2187F041287F320D90330D85BB1
:10649C00E5901313543F901766F0C2D8C2D99014EC
:1064AC00F5E0FF901766E0FD6F5403603EEF75F06A
:1064BC0004A47E00540CFFED5403FDEF4D24E3F5D2
:1064CC0082EE3414F583E0901767F06016E0FF332A
:1064DC0095E09014F38FF0124A5E9014DEE4F0A372
:0B64EC007405F0901766E09014F5F0C6
:1064F7009014DEE07002A3E0600A9014DE74FFF5EA
:10650700F0124A5E9014DEE07004A3E064016003B9
:106517000265DC9014F3E0FCA3E0FD64024C700517
:106527007F050265D212923A50047F0180027F00F4
:106537009014F3E0FCA3E0FDD39402EC6480948014
:1065470040047E0180027E00EE5F60057F070265E2
:10655700D212924450047F0180027F0012923A4087
:10656700047E0180027E00EE5F60047F09805C127A
:10657700924440047F0B8053BCFF07BDFE047F0697
:10658700804912924E40047F0180027F00C3ED9440
:10659700FEEC6480947F50047E0180027E00EE5FF3
:1065A70060047F08802512925840047F0180027F93
:1065B7000012924E50047E0180027E00EE5F60045E
:1065C7007F0A8007129258500C7F0C1287F39014A1
:1065D700F3E4F0A3F0D007D006D005D004D003D061
:1065E70002D001D000D0D0D082D083D0F0D0E0321A
:076672004405FC05090D11B0
:1053A7003EF583ECF0A3EDF0C3ED9BFDEC9AFCE931
:1053B700FF3395E0FEEF25E0FFEE33FE22ED75F0BB
:1053C7002DA424F8F582E43400F583E5822EF582D6
:1053D700E43583F58322E025E0249CF582E4340557
:1053E700F583E0FCA3E0FDEF25E02480F582E434BB
:1053F70005F583E0FEA3E0229005F9124D79901799
:105407004EE09006D1FF75F004024D44E09005F997
:1054170075F07DA42449F9740735F0FA7B01024D34
:10542700793EF583ECF0A3EDF0229006D4EF75F00A
:1054370004024D44E412499F90170DE025E024260D
:10544700F822E0FF75F005A4F58285F08312493E46
:10545700540F22EF75F005A4FF9005F9024D59741A
:10546700FFF5F0124A74FCD3E5F09400EC648094E5
:105477008022901654E09006D475F004124D44E053
:1054870022E4F0EF24FAA3F0E0FD24FCF582E434F3
:1054970005F583E022EF9006D175F004024D4490A4
:1054A7000001E92FF9EA35F0FA124AB5FFAEF0220A
:1054B7003EF583E0FCA3E0FD2274802FF58274059E
:1054C7003E222DFFEE3CFEF0A3EFF07C007D0502AF
:1054D70049C1E0FE75F02DA424E1F582E43401F51D
:1054E70083E5822F22FF901629E0FCA3E0FD22E04E
:1054F70024A3F582E43414F583E022EF25E0242683
:10550700F8760F0876FF22901629EEF0A3EFF02227
:1055170090173BE025E0FF90173AE033FE74B92F70
:10552700F582740422A804A905AA06AB07E0FEA326
:10553700E0FF22E025E02480F582E43405F583E0EE
:1055470022FFE4FCFD024CF67B017A0779499005BE
:10555700F9024D79E024DAF582E43405F58322E493
:105567007F2C7E01FDFC124CEAC3024C919017522E
:10557700E0FCA3E0FD22F583E4F0A3F0EF25E022B1
:105587009005FAE475F005124A5E90174FE004F0B3
:105597002275F02DA424EFF582E43401F583E5822A
:1055A7002F22E9D36480F8740B64809822E0FEA36D
:1055B700E0FFED25E02426F8A60608A607229017A7
:1055C70038EEF0A3EFF022901655EEF0A3EFF00DB2
:1055D700124A28901655EE2290093DE0D3648022A6
:1055E700E4F0ED75F02DA422FFE4FCFD7B1FFAF932
:1055F700F8024B74741B2FF582740622E4FCFD023B
:105607004CF674932FF582740622EF25E02426F8D2
:10561700E6FC08E622AB07AA06A905A804024CDEA9
:10562700E0A3FFE0FCA3E0FD22901644E0FF3395E2
:10563700E0FEEF2274962FF58274003E22F0AF054C
:10564700128C9BEF4E22E4F0A37405F022D3940052
:10565700EE940022124B677805124CB8AD07AC06E2
:105667002290170F124D598F827583002274002FD5
:10567700F58274002274572FF582740622745A2F0C
:10568700F58274002275F004EE124D447405F02281
:1056970025E02426F876080876002225E02426F857
:1056A700E4F608F622E0FF740BD39F222470F582FC
:1056B70074053EF58322124CF6901645024CDE9F88
:0956C700EE6480F8EC6480982286
:108C9B00AD07EDB4010F1255DF94807E0040037FCA
:108CAB0001227F0022EDB4020F1255DF94817E006A
:108CBB0040037F01227F0022EDB4030F1255DF9496
:108CCB00827E0040037F01227F00221255DF9480B9
:0B8CDB007E0040047F0180027F002229
:10962F00E4FFEF25E02400F582E4340012557D2499
:10963F00B9F582E43404F583E4F0A3F00FEFB42D11
:01964F00E139
:0196500022F7
:1092E800EF64116022EF6412601DEF641F6018EFD5
:1092F80064206013EF6428600EEF642B6009EF644C
:0C930800276004EFB42A03D38001C322C5
:109825009014A2E0FF7419D39F500BEF94265006B5
:0C983500C3EF940EFF229014A2E0FF226B
:107B8D00E4FF1254317406F00FEFB405F5E4FF7401
:107B9D00FC2F125493FE74DA2F12555EE4F0EE9022
:107BAD0006D81254A07402F09006DC12568C900682
:107BBD00E012568C0FEFB404D6E4FF74002FF5825B
:107BCD00E43406F583E4F074DE2FF582E43405F534
:107BDD0083E4F00FEFB41BE3E4FFEF25E0241BF586
:107BED0082E4340612557D2457F582E43406F5837C
:107BFD007401F0A37490F0EF25E02493F582E43442
:107C0D000612557D245AF582E43400F5837401F093
:097C1D00A3742CF00FEFB41EC19A
:017C2600223B
:10980800125611D39400EC94004005EF1256A22290
:0D9818009006D112543412564D1255022202
:1095A50012549C125466501112549C12557F125637
:1095B500144C600EEF125697221256114C6003128E
:0395C5005502222A
:02835300AE0773
:10835500C2201292E850321253C4E060291253C46D
:108365001255E72406F582E434011253D01255E77D
:10837500240EF582E434011253D01255E72411F589
:1083850082E4340180370283CC740BD39E501CEEFB
:10839500941850171253C4E0600F1253C41255E7D6
:1083A5002406F582E434018014801C1253C4E06075
:1083B50016ED75F02DA424F8F582E434001253D09F
:0C83C500E4F0AF05029808AF051295A582
:0183D1002289
:055C920090170DEFF07A
:105C9700C215C216C217E075F02DA424F8F97400D6
:105CA70035F0FA7B0190170F124D7990170DE090A0
:105CB70006D312540CE090170EF0125431E0B406DC
:105CC7000D90170EE0FF90170DE0FD02835390171C
:105CD7000E1256AC5014EF9418500FEF6411600475
:105CE700EFB41204D2178002D21630164D1256683E
:105CF70012493E601590170EE0F582758300125425
:105D07003BE6FE08E64E7002D21590170EE0240E11
:105D1700FFE433FEA3124D598F828E8312493E70E2
:105D270003025E078F828E8312543BE6FE08E64E1F
:105D37006003025E07D215025E07201703025DE9C2
:105D470090170EE064117048A3124D59900011127C
:105D5700493E701890001F12493E7010900027129C
:105D6700493E700890002A12493E6024900011E4D1
:105D770012499F90001FE412499F900027E412499F
:105D87009F90002A12543BE6FE08E64E7002D21599
:105D970090170EE064127068A3124D59900012120A
:105DA700493E701890002012493E7010900028124A
:105DB700493E700890002B12493E6044900012E45F
:105DC70012499F900020E412499F900028E412494D
:105DD7009F90002B12543BE6FE08E64E7022D21528
:105DE700801E90170F124D5990170EE0FFF5827520
:105DF700830012493E6009125668E412499FD21582
:105E070030150D90170D12540812564DEF025F0909
:105E170090170D1254081254664003025F0512547E
:105E27009CE4F0A3F030162890170EE0FF12553BC4
:105E3700FCA3E0D39400EC9400505DEF25E0249C94
:105E4700F582E434051253F8125654404D025EE1D0
:105E5700201703025EED90170EE0FF6411703DD32B
:105E67009005A3E094009005A2E09400502A9005C5
:105E7700D5E094009005D4E09400501C9005CFE045
:105E870094009005CEE09400500E9005BFE094007A
:105E97009005BEE09400400280408044EF64127099
:105EA70064D39005A5E094009005A4E09400502ADF
:105EB7009005D7E094009005D6E09400501C90051B
:105EC700D1E094009005D0E09400500E9005C1E019
:105ED70094009005C0E09400400690170DE08016EE
:105EE70090170DE0801490170EE01253EF125654DE
:105EF70090170DE04004125697221256A2229017CF
:055F07000DE01255033E
:015F0C002272
:10676F00C221EF24FA901750F0E0FF1254919017C6
:10677F004EF0128C9BEF4E60747B017A07794912B1
:10678F0053FF125466505F12549CE4F0A3F090171D
:10679F004FF090174FE0FFC39419503B1254601203
:1067AF004925540F602C9017501254F6FEF46022B6
:1067BF00EF6E701E90174FA31254D91253D5E0608D
:1067CF000302684490174FE01253EF1256544002E1
:1067DF00D22112558780BB90174E1254423021039D
:1067EF000268A00268A690174EE002687F901750CB
:1067FF00E075F07DA42449F9740735F0FA7B011296
:10680F0053FF12546640030268AB12549CE4F0A38A
:10681F00F090174FF090174FE0FFC3941950691283
:10682F005460124925540F60599017501254D912C1
:10683F0053D5E06012EE1254DB1253D5E4F012542C
:10684F000512564DEF802990174FE0FFEE12559825
:10685F001253D5E0601EEFD3940A401890174FA340
:10686F00E01255981253D5E4F012540512564DEF1D
:10687F001255032290174FE01253EF125654400255
:10688F00D22112558702682490174E12544230219C
:10689F0006760808760022E4F608F62290174E12C4
:0768AF005442760F0876FF4A
:0168B60022BF
:0959CC00901623EFF0A3EDF0F9B1
:1059D50012563425E0FBEE33FA745F2BF58274041E
:1059E5003A1253F8901639125548747B2BF5827488
:1059F500043A1253F890163D1255481255A9400322
:105A0500025C91901624E0FF648094984003025C48
:105A1500911292E85003025C91901624E0F9FB3351
:105A250095E0FAEB25E0FFEA33FE74052FF5827465
:105A3500041254B7745F2FF582740412542874212C
:105A45002FF58274041254B7747B2FF582740412F7
:105A5500542874AB2FF58274031254B774052FF5CF
:105A650082740412542874C72FF58274031254B734
:105A750074212FF582740412542874512FF5827401
:105A8500031254B774AB2FF5827403125428746D46
:105A95002FF58274031254B774C72FF5827403125D
:105AA50054281254C01253F8FF90162B125603EBCC
:105AB50025E0FBEA33FA749C2BF58274053A125300
:105AC500F8FFE4FCFD90162F124CF690162B124CA5
:105AD500DE74512BF58274033AF583EEF0A3EFF0F3
:105AE50090162F124CDEAD07AC061253B6746D2F0F
:105AF500F582740312542890162F124CDE90162B43
:105B050012561C124B67901633124CF69016331230
:105B150055665003025C9190163D124CDE90163985
:105B250012561C124B67901625124CF6901625122C
:105B350055665003025C91901639124CDE780C12B2
:105B45004CCB901625124CEA128ECD12550E90169E
:105B550024E0FF640B6004EFB4180C90163774044E
:105B6500F0A374CBF0800A9016377403F0A3743257
:105B7500F0901637E0FEA3E01254ECD39FEC9E5054
:105B850009E4901629F0A3F08015901637E0FEA3DE
:105B9500E0FFC3ED9FFFEC9E901629F0A3EFF09078
:105BA5001624E0FF640B6004EFB4180F90162AE08A
:105BB50025E0F0901629E033F08016901629E0FED6
:105BC500A3E0FF1254D212550E7D031249D312558C
:105BD5000E901624E01253B71256743E1253F81263
:105BE50055EF90162912552CE4FCFD12565B9016C4
:105BF50024E01253B71256741254281256743E12EA
:105C050053F8FF901629EEF0FCA3EFF0FD7B907A98
:105C150001901623E0F91253B712567C3E1253F841
:105C2500C39DEE9C50111254ED1253B612567C12C0
:105C350053A71255FB80271253B61255FB3E12533C
:105C4500F81254ECC39FEC9E50171253B61255FB35
:105C5500125428ED2BFDEC3A1253B512567C125412
:105C650028901623E0FD1253B71255FB3E1253F848
:105C7500FF12550ED394FFEE940F400A9016297427
:0C5C85000FF0A374FFF09016291255B424
:015C910022F0
:0570D100901641EFF0F4
:1070D600AF05EF1253B81254C0F583E0FFA3E0905A
:1070E600164DCFF0A3EFF0AF03EF1253B81254C012
:1070F6001253F8FF90164EE02FFF90164DE03EFE1D
:10710600E4FCFD90164F124CF6E47F1EFEFDFC904B
:10711600164F12556D50030271DB90164DE0FEA31B
:10712600E0FFE4FCFD780C124CCBA3124CEA128E65
:10713600CD901649125603901649124CDE780C1261
:107146004CCB901649124CF61256307802C333CE09
:1071560033CED8F91256B3124CDEE47B3F1255F506
:107166007806124CB8C004C005C006C00790164980
:10717600124CDE7806124CB8D003D002D001D000F3
:10718600124B679016451256BDC004C005C006C016
:10719600071256307802C333CE33CED8F91256B31F
:1071A600D007D006D005D0041256BDE42FFFEE342A
:1071B60008FEE43DFDE43CFC780C124CB8D3EF9499
:1071C600FFEE940F40047E0F7FFF9016411254424B
:0571D600A60608A60753
:0171DB002291
:1093E4007C007D0B1249C1EEA2E713FEEF13FFC30D
:1093F40094CBEE648094845005E4FEFF80087435B9
:079404002FFF74FB3EFE2266
:0B90120090173AECF0A3EDF01255C5EA
:10901D001293E41255C51255173E1253F81255EF1F
:10902D0090173812552CEE3395E0FDFC12565B125D
:10903D0055171254281255243E1253F8FF1255C5D8
:01904D002200
:0D785700901751EFF0A3ECF0FEA3EDF0FF51
:10786400AC02AD03129012901752EEF0FCA3EFF0AD
:10787400FD7B2C7A01901751E0F91253B71256840C
:107884003E1253F8C39DEC6480F8EE648098501166
:107894001255741253B61256841253A71256098005
:1078A400281253B61256093E1253F8FF125574C3E8
:1078B4001256C650171253B6125609125428ED2BFD
:1078C400FDEC3A1253B5125684125428901751E025
:1078D400FD1253B71256093E1253F8FF901752EE99
:1078E400F0A3EFF0D394FFEE6480948F400A9017D6
:0E78F40052740FF0A374FFF09017521255B4A7
:017902002262
:02790300A907D2
:10790500E4FBFAE9FD3395E0FCED25E0FFEC33FE01
:1079150012563BF583E020E4030279A11255A950E4
:1079250025E964809498501EED25E0FFEC33FE7444
:107935009C2FF58274051254B71254C01253F82DBA
:10794500FFEE3CFE800A1253B61254C01253F8FFE4
:107955001293E4AA06AB071253B674162FF5827478
:10796500053E1253F8D39BEE9A50317C007D05AF4E
:1079750003AE021249C1AA06AB07EAC313FAEB1319
:10798500FBD394FFEA940F40047A0F7BFFAD0312FB
:1079950053B612563BF583EAF0A3EDF0AF01EF12B3
:0979A50053B812563B1253F8FFCF
:0179AE0022B6
:105F0D00EF24FA90165912548E04901654125644DA
:105F1D007003025FDC12554F9016591254F690160D
:105F2D0053F0F47003025FBFE0FF64117003026170
:105F3D007FEF6412700302617F12546075F005EFFC
:105F4D0012544E700302617F9006ECE0FF901657DD
:105F5D00F0BF020B901654E0FF901653026028908C
:105F6D001657E0B40406901653026036901657E0AB
:105F7D006403600302617F9016531256AC5013EF09
:105F8D009418500E1253DD9016551254C91255CE59
:105F9D00800D90165312553AFFA3E0901655CFF091
:105FAD00A3EFF0901654125627901653E0FB7A008B
:105FBD00801A9006ECE06403600302617F90165432
:105FCD00E0FF901653E0FB7A00E4FDFC0278579059
:105FDD00165912541390165912555BE0901658F03D
:105FED00129825901653EFF06411700302617FE053
:105FFD00FF6412700302617F12546075F005EF1299
:10600D00544E700302617F901654E0FF9006D41237
:10601D005435E0901657F0B40206A3E0FD0259CCBA
:10602D00125479B40414901658E0FF1279039016A7
:10603D0054125442A60608A607221254796403602E
:04604D000302617F6A
:1060510090165BF0A3F0A3F0A3F0901659E0900521
:1060610013125417E490165AF090165AE0FFC364C5
:106071008094994003026129900513124D59EF3321
:1060810095E08F82F5837405124D3312493E540F0A
:05609100700302612014
:1060960090165AE0FD1253B71254C0F583E0FFA3E1
:1060A600E090165FCFF0A3EFF0ED1255AA503290B4
:1060B600165AE0FF648094985027EF1253B8749CE8
:1060C6002FF58274053E1253F8FF901660E02FFFFD
:1060D60090165FE03EFE9016551254CE1255CE80B5
:1060E6000B90165FE0FFA3E0901655CFF0A3EFF0FC
:1060F60090165BE0FEA3E0901655125629D3125671
:10610600C6401790165BECF0A3EDF090165AE0FE31
:0A6116003395E090165DF0A3CEF083
:1061200090165AE004F002606A901654E0FF901650
:106130005BE0FCA3E0FDA3E0FAA3E0FB127857309C
:10614000013DE490165AF090165AE0FFC364809423
:10615000AD502AEF3395E0FE74A92FF58274143EFA
:10616000F583E0701090165AE01253B81254C0F53F
:0F61700083E4F0A3F090165AE004F080CAC20155
:01617F0022FD
:1080300090173E125488240290173D125644603225
:1080400012554F90173F1254F6FFF4606D90173C95
:10805000EFF012546090173C125449605D12545A6C
:108060001254A6128D76EF7802C333CE33CED8F9F0
:10807000803C90173F12541390173F12555BE090CD
:10808000173EF012982590173CEFF01254609017AD
:108090003CE012544B602390173EE012545B1254A4
:1080A000A6128D76EF7802C333CE33CED8F9FF9087
:0A80B000173D125442A60608A60769
:0180BA0022A3
:1073CA009017421254882403901741125644604F72
:1073DA0012554F9017431254F6FFF470030274913A
:1073EA00901740EFF09006F4E0640570271254609D
:1073FA00901740125449700302749112545A900023
:10740A00031254A9128D76EF7802C333CE33CED845
:10741A00F9027479901741E0FF90174002748C903A
:10742A00174312541390174312555BE0901742F01A
:10743A00129825901740EFF0125460901740E0120E
:10744A00544B604390174112547C6405702E901778
:10745A0042E012545BE92FF9EA35F0FA9000031280
:10746A0054B0128D76EF7802C333CE33CED8F9FFFB
:10747A00901741125442A60608A60722901741E027
:07748A00FFA3E0FD1259CC45
:0174910022D8
:057CC000901712EFF027
:107CC5009006D3125480901716F012982590171528
:107CD500EFF0901712E0FF12547DB40208901716CA
:107CE500E0FD0259CC90171212547CB4041B901776
:107CF50016E0FF901715E06F705812790390171270
:107D0500125442A60608A607229017161256AC5022
:107D150020EF9418501B1253DD9017131254C9907D
:107D25001713EEF0A3EFF00D1249D3901713EE8061
:107D35000D90171612553AFFA3E0901713CFF0A335
:107D4500EFF0901712125627901716E0FB7A0012E3
:027D550078575D
:017D57002209
:108D76007C007D6A124DDA901744124CF690174427
:108D8600124CDEE47B64FAF9F8124BFF901744129A
:108D96004CF6E47FFF7E0FFDFC901744124CEAC3AD
:108DA600124CA7400A901744124D0200000FFF9084
:058DB6001744124CDE21
:018DBB002295
:089C08000020406080A0C0FFB5
:0D9B34007F147E00EF1F70011EEF4E70F7D2
:019B41002201
:109AA8007F381296F47F061296F47D0EE4FF029B2F
:019AB8007538
:0596F400901780EFF06B
:1096F900A2AF9222C2AF129694EF20E7F990178099
:09970900E0FF125021A22292AFF0
:019712002234
:10969400A2AF9223C2AF75A0FFC2B5D2B6D2B712A1
:0F96A4009B34ADA0C2B7129B34A22392AFAF0587
:0196B3002294
:059C6E007F010296F4E5
:10502100A2AF9224C2AF8FA0129B34C2B5C2B6D236
:0D503100B7129B34C2B7129B34A22492AF79
:01503E00224F
:10985D00A2AF9225C2AF8FA0C2B6D2B7D2B5129B1E
:0A986D0034C2B7129B34A22592AF5B
:0198770022CE
:0C9B7500901781E05FF04DFFF00296F4C5
:02997900AC0739
:10997B00A2AF9226C2AF129694EF20E7F9AF041272
:06998B00985DA22692AFD8
:0199910022B3
:1094EF00901754124D79901754124D591249256007
:1094FF0013901754E475F001124D62124925FF12B3
:05950F00997980E222C1
:069088009016F5124D796F
:10908E00A2AF9227C2AF129C6EE4FDFF129B81909D
:10909E0016F5124D591294EFE4FD7F01129B81904B
:1090AE0016F8124D591294EF7D107F01129B81A27A
:0390BE002792AF47
:0190C100228C
:0C9B8100EF75F040A42D2480FF0296F444
:0B9BBB00E4F584EF909C0893F5D322A2
:04667900410BB10020
:107C270090168BE0FF75F07090B401124D44EF256C
:107C3700E02583AF8222E475F001124A5E90168D2B
:107C4700E475F001024A5EFE7A0679D17B0190164F
:107C5700DA7402F0A37470F022AFF0FEE0FCA3E048
:107C6700F5828C83E493FD22901687F0A3EFF0E46E
:107C770090168DF0A3F0227E007C027D701249C120
:107C870074012FF974B43EFA7BFF22EFF0A3EDF0F5
:107C9700A3EBF0A2AFE433A3F0C2AF2275F070EE0E
:107CA70090B401124D44EE22E475F001024A74FDCE
:097CB700EDFFEEF0A3EFF0E42272
:069C5600E4900BB1F022C6
:079C1000900BB17401F0227A
:0591D400901768EFF0A8
:1091D900129C00E4901769F0901768E0FFA3E0FE85
:1091E900C39F5014127CA3127C36127C4E1290FC41
:0B91F900901769E004F080E002945938
:108B1E0090176A7402F0E4A3F0129C007EB47F00FA
:108B2E007A17796A128B5D7EFF7F917A17796B12B5
:108B3E008B5D1294597E027F707D007B017A0679DF
:0F8B4E00D1124E07127B8D1299AB7F1E0291D46C
:0E8B5D007B019016DAE4F0A304F01290FC22E3
:1098E00090FF91E493F4600990B400E49364026003
:0A98F00003128B1EE49006CFF02255
:109A200030030E201A10900BB1E07002D206D21A49
:079A300022D2021272E122B2
:03501B00029A20D6
:0A9514009006CFE0FFC3941E50182C
:10951E009006D3E0901782F0127C7E78D17C067D87
:08952E00017E027F701248FF6C
:03953600C21A2234
:109841009006CFE0C3941E5012129C009006CF12D6
:0C9851007C2A127C4E1290FC12945922CA
:1099AB00A2AFE433901783F0C2AF129841C21A9062
:0799BB001783E024FF92AFC7
:0199C2002282
:087DF00090166EEDF0A3EBF01C
:107DF800A3E004F0901673EFF0A3EBF090166EE09A
:107E0800FF901673E0FED39F505B127CA3127C3662
:107E1800901675F0A3EFF0901674127C2A901677DE
:107E2800F0A3EFF0E4901671F0A3F0901677127CAF
:107E3800AF901675127C60128549901675127C47B2
:107E4800901671127C47C3901672E0947090167168
:107E5800E0940240D6129459901673E004F0A3E01F
:107E680004F0027E049006CFE0FF90166FE0D39FE7
:0B7E78005009A3E0C39F4003129514C3
:017E830022DC
:0F6EA000901685EDF0901684EFF0901686EBF0CB
:106EAF0090168BEFF0A3EBF0901685E0FF90168B0A
:106EBF00E0D39F4003026F75A3127C2A127C6F9060
:106ECF00168DE0FEA3E0FFC39470EE9402501A906B
:106EDF001687127C6374412FF58274093EF583ED9A
:106EEF00F0901687127C3D80D6127C27901689F081
:106EFF00A3EFF090168C127C2A127C6F90168712DB
:106F0F007CAF901689127C60128549901689127C8D
:106F1F003DC390168EE0947090168DE0940240DC85
:106F2F00127C27901689127C7290168DE0FCA3E0DC
:106F3F00FDC39470EC9402501D901689127CAFAF74
:106F4F00F0FE74412DF58274093CF583E0FD128546
:106F5F0049127C4480D312945990168BE004F0A30D
:106F6F00E004F0026EB79006CFE0FF901686E0FEC9
:106F7F00D39F5020901684E0FDA3E0C39DFDE494C1
:106F8F0000FCEE7A002DFDEA3CFCC3ED9F7480F807
:106F9F006C9850139006CFE0FF901684E0D39F506B
:0A6FAF0009A3E0C39F4003129514EC
:016FB90022B5
:03814300901699FA
:10814600127C9212501290169AE0FE901699E090C8
:1081560016A1127CB690169DF090169BE0FF901625
:10816600A1E0FCA3E0FD7B017A0979419016BB12E0
:108176007C5812960D9016A1740275F070124A5E24
:1081860090169DE0FF127C7EA3124D79129C009002
:10819600169E124D59AE02AF017A097941127C53EF
:1081A6001290FC12945990169DE004F0E0C3941EC0
:1081B60040A79014D6E0FF129B4F90169CE024FF38
:0281C60092AF76
:0181C8002294
:0385C0009016AC66
:1085C300127C921250129016ADE0FE9016ACE09021
:1085D30016B1127CB69016B0F09016B0E0FFC394BB
:1085E3001E503E75F070EF127C2FFE9016B3F0FA1A
:1085F300A3EFF0FB9016AEE0FF9016B1E0FCA3E012
:10860300FDA9037BFF9016C3127C581298C69016DF
:10861300B1740275F070124A5E9016B0E004F080F7
:10862300B89014D6E0FF129B4F9016AFE024FF9250
:01863300AF97
:018634002223
:109AB900FFE475F001024A5EE0FEA3E0F5828E83C1
:019AC900227A
:108E01007E107FAB900FB8EEF0A3EFF0900FB4EEB1
:108E1100F0A3EFF07E117F73900FBAEEF0A3EFF0A5
:108E2100900FB6EEF0A3EFF0E490123BF0C2287E73
:108E31000F7FBC901086EEF0A3EFF0901084EEF05F
:048E4100A3EFF02289
:03500F00027E849A
:107E8400C0E0C0F0C083C082C0D075D000C000C0C4
:107E940004C006309825C298900FB4129AC1E5998F
:107EA400F0900FB4129ABAFCE5F0B4730EECB4116E
:107EB4000A900FB47410F0A374ABF030994190128F
:047EC4003BE0603708
:107EC800900FBA129AC1E0901784F0C299F5999070
:107ED8001088E599F090123BE014F0900FBA129ACE
:107EE800BAFCE5F0B43B14ECB41210900FBA74115C
:057EF800F0A37473F01B
:107EFD008004C299C228D006D004D000D0D0D08240
:077F0D00D083D0F0D0E03278
:1098FA00900FB8E0FEA3E0FF900FB4E06E7003A3F0
:0A990A00E06F60037F01227F00225E
:10953900900FB8129AC1E0900FB8129AB9900FB86B
:10954900E0B4110FA3E0B4730A900FB87410F0A33C
:0395590074ABF000
:01955C0022EC
:03503F000287895C
:10878900C0E0C0F0C083C082C0D075D000C000C0B6
:1087990004C006C00730983AC298901084E0FEA33E
:1087A900E0FFF5828E83E599F08F828E83E0648EF7
:1087B90060069014DA7407F0901084129ABAFCE5F6
:1087C900F0B4840EECB4100A901084740FF0A37402
:1087D900BCF0309902C299D007D006D004D000D09D
:0A87E900D0D082D083D0F0D0E0326F
:10991400901086E0FEA3E0FF901084E06E7003A335
:0A992400E06F60037F01227F002244
:10955D00901086129AC1E0901086129AB9901086DA
:10956D00E0B4100FA3E0B4840A901086740FF0A33A
:03957D0074BCF0CB
:0195800022C8
:106180004C00500049002000540043560050756CEC
:106190007320313A2573257320323A257325730015
:1061A000333A2573257320343A2573257320353A05
:1061B000257325730043562031303A25732573200B
:1061C00031313A257325730031323A257325732016
:1061D00031333A2573257331343A257325730043DF
:1061E0006F6E747261737420256420006F666600A0
:1061F000363700363738003637383900506F6C790B
:1062000070686F6E792025732000526973696E671C
:106210000046616C6C696E6700547269616E676CF0
:10622000650052616E646F6D0053706972616C003D
:106230002030002E35002031002032002033002095
:106240003400203600203800313000313500323043
:1062500000323500333000417270656767696F2026
:1062600025733A202573004B59006B790043563A49
:10627000252D33642054723A25642025632564005B
:10628000506174726E3A202573004661646520691E
:106290006E3A2573206F7574257300526164696FBF
:1062A0003A25642025733A25732025732000435630
:1062B000313A252D3364204356323A256420004379
:1062C00056313A252D3364204356323A2573200047
:1062D0006C6F6300FF618002FF618203FF618404D1
:1062E000FF618600FF618806FF618A05FF61800209
:1062F000000600070008000900050009000D001154
:106300000007FF9C730008FF9C62000CFF9C780054
:106310000DFF9C3A0102FF9C7D0103FF9C41010798
:10632000FF9C820108FF9C48010CFF9C87010DFF28
:106330009C4F0006FF6B250008FF99C3000BFF91DF
:10634000A1000DFF7F140105FF8C04010DFF82D217
:106350000006FF9C8C0007FF9C17000CFF9C91001F
:106360000DFF9C1E0103FF9C960104FF9C25010963
:10637000FF9C9B010AFF9C2C010EFF9CA0010FFFBC
:106380009C330009FF99920109FF9992000AFF933B
:1063900014010AFF9314000AFF99C3000DFF80BB8C
:1063A0000104FF83D2010AFF9673010DFF7492006E
:0E63B00007FF93920108FF9713010FFF97322A
:10667D004112CC004112CD004112D3004112D40081
:10668D004112D5004112D6004112D9004312E20049
:10669D0000004113CE024113D3014113A40059133D
:1066AD00716162636465666768696A6B6C6D6E6F54
:1066BD007071727374757677787959138A41424384
:1066CD004445464748494A4B4C4D4E4F5051525305
:1066DD005455565758594113A3004313E9011371EB
:1066ED004113D8004113CB004113E7024112EA00D8
:1066FD004113D9004113E8004113E632411414004F
:10670D0048127F00FA00FA00FA00FA4113D4000C87
:10671D0009FF61ECFF61F0FF61F3FF61F74F13ECCF
:10672D00FF620AFF6211FF6219FF6222FF62296098
:10673D002712A5FF6230FF6233FF6236FF6239FF19
:10674D00623CFF623FFF6242FF6245FF6248FF62AB
:10675D004BFF624EFF6251FF6254010801021500AA
:01676D00012A
:1056D000EDFF3395E0FE75F003EF124D44EE75F0EB
:1056E00003A42583F583227A1379BA9016F87B01F7
:1056F000124D797A1379A72224719013E97B01F96D
:10570000E43413FA024D7990128775F003ED124DCF
:1057100044EC22EFF0A2AFE433A3F01295C8C2AF7D
:105720009013D47401F0EF75F005A4FF9012E2021B
:105730004D592471F9E43413FA124D790249257B4D
:10574000FF9015DB024D79901414E025E0247FF5DD
:1057500082E43412F583229013A4E075F07DA42432
:1057600049F9740735F0FA7B019012E2024D791283
:105770004D59124D8E9015DE124D797B01229013FA
:10578000E9124D59901371C3E99582EA9583222459
:105790008AF9E434139013E9FA7B01024D799013EE
:1057A000E9124D590249259013A4E075F002A4FFB7
:1057B000AEF024F0F974623EFA7BFF9012EC124DC9
:1057C0007974F82FF974623EFA9013D522FD901384
:1057D000D5124D59124A8AAEF07802227BFF9013FF
:1057E00003024D797B019012E5024D79901709E093
:1057F000FFA3E0CF9015DEF0A3EFF022124D591277
:105800004D8E9015E4024D799016C6124D597402D2
:1058100012498D7BFF7A6279D422E02471F9E43455
:1058200013FA229016CF124D5990000322FF9012C6
:10583000CEE04EFEA3E04FFFEE9012CEF0A3EFF0CD
:105840002274FB2FF582E43413F583229012D002E8
:105850004D79901306024D79EDFF3395E0FE2275E8
:10586000F005EFA429F9EA35F0FA0249259013E989
:10587000024D59740312498D7BFF7A6279D822EF69
:10588000F09012EC124D59024A8AE075F003A424FC
:10589000A5F582E43412F583024D597B01E0FD90B9
:1058A000171B229013D3F07BFF22D3EF64809480E8
:1058B000229015E1024D79124D59124D8E9015EA44
:1058C000124D797B012275F003A424DAF582E434C9
:1058D00013F5832275F005A4240BF582E43413F547
:1058E000832275F005A42409F582E43413F583229C
:1058F00075F005A4240AF582E43413F58322E0FE52
:10590000A3E090128775F00322C39014D8E094109E
:105910009014D7E09427229012D0124D59EB8A832D
:1059200089827BFF22901757E4F0A3227BFF7A62E3
:1059300079DC22124AB5FFAEF0D39400EE94FE2239
:105940007B017A1379BA22E025E0243EF582E43423
:1059500012F58322EFF0D36480948022901757745D
:10596000FFF0A32290093DE0C3648022E49013A3DA
:10597000F07F03227B01E0FD90171B740DF022E005
:1059800024FF92AFE49013D4F0229015ED124D79DC
:105990007A1379BA22E025E02406A3F0229013D3EB
:1059A000F07BFF2224D4F58274063EF58322124D4B
:1059B0005974019013826B22124D59740190138314
:0C59C0006B2224D8F58274063EF5832289
:1086A9007F199013FBE4F0A3DFFC7B017A0779497A
:1086B9001257697BFF7A6279F09012EC124D797A40
:1086C9006279F89013D5124D7912579E9012EFF0F6
:1086D900E4A3F090136DF0FF125813EF1258C6126D
:1086E9004D790FEFB404F1E49013A6F09013B9F0AB
:1086F9009013CDF09013D0F09013D2F09012D8F0DF
:108709009012DBF09012DDF09012DFF09012E1F0A0
:01871900223D
:069C5C00E49012EBF0227F
:10885C0090176CEEF0A3EFF0AF051DEF605390177F
:10886C006CE0FEA3E0F5828E83A3A3124D829012DE
:10887C00EBE0FF1258D4124D7990176CE0FAA3E09C
:10888C00FBF5828A83E493FEEF1258E2EEF08B82C2
:10889C008A83740193FF9012EBE01258F0EFF09082
:1088AC0012EBE004F090176CE475F005124A5E8050
:0288BC00A722F1
:10940B009012E51257A1FE1258E2E0FFEE1258F04F
:10941B00E0FD129B819012E51257A11258D4124D08
:07942B0059901300024D7976
:1097CD009012E5124D59740112496B9012E5125722
:0E97DD00A1FF9012EBE0B50704E412498D22C3
:10936900D3ED6480948040047401800274FF124933
:109379006B124925FFB4FF03E4800A90171BE0FE36
:09938900B50705EE1412498D220E
:109992007B017A1379CEAD0790171B7408F01293EE
:0999A200699013CEE0FF029BBBAB
:109314007B017A09793DAD0790171B7404F0129311
:1093240069E49013A4F0E075F07DA42449F974076E
:0C93340035F0FA1257691257A7024D7964
:0580BB0090176EEFF0CC
:1080C000E49013A3F01293BB12577E401512586D23
:1080D000D3901389125788500912586DC3E99471CF
:1080E000800712586DC3E9948A90176FF090176E4D
:1080F000E0FED3648094804019A3E0FF12578FE420
:10810000D39F5026EFC3941950201258417401F0A8
:10811000801890176FE0FF1256F8E4D39F500BEFD2
:10812000C394195005125841E4F090176FE0FFD343
:10813000EE6480948040047D0180027D00129A8666
:0381400002501BCF
:1083D200901497E0FEE4D39E5074EEC39419506E4D
:1083E200EF124DAE8402018412028422038432040D
:1083F200843AFC842AFD841AFE840AFF0000844029
:1084020090178574A0F0803690178574A4F0802EA2
:1084120090178574A1F0802690178574A5F0801EB0
:1084220090178574A2F0801690178574A6F0800EBE
:1084320090178574A3F0800690178574A7F09017A3
:0E84420085E0FF129262901497E0FF129262A2
:018450002209
:10939200901786EFF0BF01047FB48009901786E032
:1093A200B4FF057FB51292627A1279EA901786129B
:0993B200589B7405F01293692226
:1096730090178712595440047FB280027FB312922D
:10968300627A14791490178712589B7404F002932A
:01969300696D
:10749200EF124DAE74B20174CB0274E30374FB04B9
:1074A2007507FC74EFFD74D7FE74BDFF0000751103
:1074B20012592504F0A374A8F0805474FF90175752
:1074C200F0A3F0A374ACF080461259257410F0A317
:1074D20074A9F0803A12595C74F0F0A374ADF08094
:1074E2002E1259257440F0A374AAF0802212595C1E
:1074F20074C0F0A374AEF08016125925747FF0A305
:1075020074ABF0800A12595C7481F0A374AFF090EE
:107512001759E0FF129262901757E0FEA3E0FF9026
:107522001414E0FD12574BEE8FF0124A5EED125723
:107532004BE0FEA3E0D394F4EE9401400CED12571D
:107542004B7401F0A374F4F022C3EE94005008EDE2
:0775520012574BE4F0A3F017
:01755900220F
:1097130090178812595440047FB680027FB7129283
:0F972300627A1379D990178812597412936922B8
:1097320090178912595440047FB880027FB912925F
:0F974200627A1379E89017891259741293692289
:099BEE009012D0124D59024DD421
:1096B4009013D37401F07A9679511257DC7A847935
:1096C400CD12584C7A9679D41258527F01029BD00D
:1096D4009013D37402F07A9679B41257DC7A4E79E7
:1096E4003C12584C7A9779511258527F02029BD0FF
:1097510074031258A37A9679D41257DE7A7F79A3CB
:0F97610012584C7A9779701258527F03029BD09E
:1097700074041258A37A9779511257DE7A8C79E6DD
:0F97800012584C7A97798F1258527F04029BD05F
:10978F00740512599D7A9779701257DE7A8E7989FE
:0F979F0012584C7A9779AE1258527F05029BD020
:1097AE00740612599D7A97798F1257DE7A6D797AEF
:0F97BE0012584C7A9679511258527F06029BD05E
:109651009013D37407F07BFF7A9779AE1257DE7AB5
:1096610086793512584C7A9679B41258527F07028E
:029671009BD08C
:028E4500AD0777
:108E4700ED3395E0FEEF7802C333CE33CED8F92465
:108E570000F974073E9016FB125798AF05EF33954C
:108E6700E0FE9012521256D6124D599016FE124D30
:108E7700799016FB1257A1B40205740312498D02AB
:028E8700501B7E
:108FD5001258AA7BFF40067A6279E480047A6279A6
:108FE500E09012F11256D0124D791258589012F1A4
:108FF5001256D612582612493EFCEF7802C333CEDC
:0D90050033CED8F91259A4ECF012501B2202
:059C7300E4FD028FD5A5
:059C78007D01028FD503
:059C7D007D02028FD5FD
:059C82007D03028FD5F7
:059C87007D04028FD5F1
:10824F009016C6124D791258AA40289016C612578A
:10825F00A124FE600A146009146008240470618070
:10826F002680009016C6124D59740412498D12596A
:10827F002C80479016C61257A124FE600F14601170
:10828F0014602E24047039125873802E12580880EF
:10829F00299016CCE075F003A42478F582E434120B
:1082AF00F5831257A1D3648094EB401412580880C1
:1082BF00099016C6124D591258739016C9124D795E
:0382CF0002501B3F
:028B6B00AC0755
:108B6D00125858EF7802C333CE33CED8F92400F91A
:108B7D0074073EFA7B01901701124D7912585890E7
:108B8D0012521256D6124D59901704124D79AF0448
:108B9D00901704124D599016C9124D799016CCEDBF
:0A8BAD00F0901701124D5912824F8B
:018BB700229B
:059C8C007D0A028B6B54
:059C91007D0B028B6B4E
:059C96007D0C028B6B48
:059C9B007D0D028B6B42
:059CA0007D0E028B6B3C
:10755A001258AA40431257071256DEA3E475F001E7
:10756A00124A5E30297C1257071256DE1259AE7043
:10757A0008E965827003EA65836015125707125697
:10758A00DE1259B87008E965827003EA65837052A1
:10759A007B017A13798480411257071256DEA3744D
:1075AA00FFF5F0124A5E3029391257071256DE12D9
:1075BA0059AE7008E965827003EA6583601512574F
:1075CA00071256DE1259B87008E965827003EA6537
:1075DA0083700F7B017A1379811257071256DE12D4
:1075EA004D791257071256DE124D59D3901389124C
:1075FA00578840087B017A1379898011125707123C
:10760A0056DE125781500F7B017A13797112570790
:07761A001256DE124D792229
:1090C200901770ECF0A3EDF0C22912755A90177048
:1090D2001258FE1256DA124D59C3E99471FD9017D7
:1090E20070A3E07802C333CE33CED8F924D3F5820D
:0A90F20074063EF583EDF002501BFA
:1088BE00901772ECF0A3EDF0D22912755A90177240
:1088CE001258FE1256DA124D59C3E99471FD9017E3
:1088DE0072E0FAA3E0FB7802C333CE33CED8F9248C
:1088EE0013F58274073EF583EDF0125902EB124D2B
:1088FE0044EA1256DE1257A1C3648094EC500B90DA
:0D890E001772A3E02405FF128E4502501BD6
:079C17007D057C000288BE00
:079C1E007D067C000288BEF8
:079C25007D077C000288BEF0
:079C2C007D087C000288BEE8
:079C33007D097C000288BEE0
:069C6200E4FDFC0290C2CB
:079C3A007D017C000290C2D5
:079C41007D027C000290C2CD
:079C48007D037C000290C2C5
:079C4F007D047C000290C2BD
:106B25001258AA5003026BBB12572C7401900749E7
:106B35006B7008E965827003EA6583702090093DF2
:106B4500E014601214601114601024037062901335
:106B5500A47401F0805A801A8035E4804F12572CB6
:106B650074019007C66B7008E965827003EA658356
:106B750070089013A47402F0803612572C7401909B
:106B850008436B7008E965827003EA6583700890B5
:106B950013A47403F0801912572C74019008C06B6C
:106BA5007008E965827003EA658370049013A4F0A8
:106BB500125757026C4612572C74019007496B7097
:106BC50008E965827003EA6583700F12596494833E
:106BD50050439013A47403F0806712572C740190EE
:106BE50007C66B7008E965827003EA6583700280E9
:106BF5004C12572C74019008436B7008E96582703C
:106C050003EA65837012125964948150089013A4A5
:106C15007401F0802CE4802512572C74019008C073
:106C25006B7008E965827003EA6583701412596414
:106C3500948250089013A47402F08005E49013A484
:0B6C4500F01257571257A7124D79228A
:1099C3001258AA40079013A37401F02212596C1283
:0899D300928F7F391299DB220B
:1095C80012577E401512586DD39013891257885040
:1095D8000912586DC3E99471FF2212586DC3E994BA
:0395E8008AFF22D5
:0291A100AE0717
:1091A3001295C8D3EE648094804012748A2F1257AC
:1091B3009112572C12585F54F04401800E74712F92
:1091C3001256FA12572C12585F54F012498D02505E
:0191D3001B80
:037F140090178A39
:107F170012587F24FAFFE5F034FFFE90178AE0D36A
:107F2700648094809013DA75F003EF400A1256DAF2
:107F3700A3E475F00480091256DAA374FF75F0FC08
:107F4700124A5E9013DA1256D6124D59D39062DC5C
:107F5700125788400C12592C9013DA1256D6124D2C
:107F6700799013DA1256D6124D599062D412578768
:107F7700500C1258139013DA1256D6124D799013EB
:107F8700DA1256D612582612493E1257CDC333CEAF
:0C7F970033CED8F91259C2EDF002501B95
:108BB800EF124DAE8BD8018BE2028BEC038BF604DF
:108BC8008BFBFC8BF1FD8BE7FE8BDDFF00008C003F
:108BD8007E007F01227EFF7FFF227E007F10227EA3
:108BE800FF7FF0227E007F40227EFF7FC0227E0032
:0C8BF8007FFF227EFF7F0122E4FEFF22AF
:038C040090177452
:108C0700125713E92FF9EA35F0FA901774E0FF12BB
:108C17008BB8900001EE8FF0124AED9000011259C7
:108C2700334008900001E4F5F08011C3EF94C6EEDD
:108C37009403400B900001740375F0C6124B3A126F
:088C4700501B90177512597FB4
:018C4F002202
:0382D2009016CD36
:1082D500125713E92FF9EA35F0FA9016CF124D79B6
:1082E5001257CEC333CE33CED8F924DDF974063E0A
:1082F500FA7B019016D2124D799016CDE0FF128BC4
:10830500B8125823EE8FF0124AED9000031259333C
:108315004013125823E4F5F0124B3A9016D2125836
:10832500267402801CC3EF94C6EE9403400B1258CA
:1083350023740375F0C6124B3A9016D21258267460
:0D8345000512499F12501B9016CE12597F51
:018352002208
:107D5800900727E024719012961256FD124925903B
:107D680012D7F090072BE024719012991256FF1247
:107D780049259012DAF090072FE090129C125732A2
:107D88009012DCF0900733E090129F125732901255
:107D9800DEF090073712581A9012A2125739901233
:107DA800E0F0E4FD125858EF7802C333CE33CED852
:107DB800F92428F58274073EF583E0601024FD60FD
:107DC8000C14600E24027019125813800812587887
:107DD800800312592C1258589012701256D6124D10
:077DE800790DED640570BD8B
:017DEF002271
:1084CD001281C97A61798D12573F9012F112576F4F
:1084DD007A1379A51258B19012F41257FC7A1379C8
:1084ED00B89015E71256EE1250A77A6179A012577F
:1084FD003F9012F712576F7A1379CC1258B1901230
:10850D00FA1257FC7B017A1379CF9015E7124D794A
:10851D009012FD1258B77A1379D112598A1250A7B9
:10852D001256E7129088129C5C7E637F007D0A12C2
:0C853D00885C7A1279CC1257E402940B8F
:107FA30012596C12928F7F391299DB127D587BFF25
:107FB3007A6179B512574190127012576F7A12791C
:107FC300D71258B19012731257FC7B017A1279DAE7
:107FD3009015E71256F01250A77BFF7A6179C81209
:107FE300574190127612576F7A1279DC1258B1907A
:107FF30012791257FC7B017A1279DE9015E7124D44
:108003007990127C1258B77A1279E012598A125079
:10801300A71256E7129088129C5C7E637F507D0AFC
:0D80230012885C7A1279D31257E402940B94
:108CE6007BFF7A6179DF1257419013CEE0FFE412E1
:108CF60057F47B017A1379A71250A77BFF7A617923
:108D0600861257411259401250A71256E712908800
:108D1600129C5C7E637F827D0112885C7B017A12E5
:088D260079D41257E602940B08
:108E89007BFF7A6179FC12574190093DE075F00347
:108E9900A42409F8124D501257757A1379A7125064
:108EA900A7E49013BAF01256E7129088129C5C7EE0
:108EB900637F8C7D0112885C7B017A1279D5125708
:048EC900E602940B1E
:106D7A009013A3E0600D7F0312928F7F381299DB84
:106D8A00128D2E9012D6E0B40205E49013A3F0906F
:106D9A001497E0FF6411600BEF64126006EFC3946E
:106DAA0019400890123CE0901497F0901497E0FF75
:106DBA00E4D39F4003026E76EFC394194003026E38
:106DCA0076125841E09014976009E0248AF9E43475
:106DDA00138007E02471F9E4341312579512579E71
:106DEA009012EFF07BFF7A6279571257419013A302
:106DFA00E060067A62796780067BFF7A62796A12B6
:106E0A0057757A1279EF9015E11256F01250A712BF
:106E1A005747E0FEA3E02406FFEE34FFFE129B99DB
:106E2A009015E3EEF0A3EFF07BFF7A62796D1257CB
:106E3A00419014971259471257EF901414E0FF2407
:106E4A0001FCE4339015E0F0A3CCF0EF12574BE0CD
:106E5A00FEA3E0C394FAEE940050047F2D80027FD3
:106E6A00209015E2EFF01259401250A7125909402A
:106E7A000D1256E7129088E49014D7F0A3F0129CF2
:106E8A005C7E637F967D0512885C7B017A1279D6D7
:066E9A001257E602940B02
:1086350012596C12928F7F391299DB7BFF7A62791E
:10864500801257419012EAE075F003A424ECF582FC
:10865500E43413F583124D591257757A1379A7121D
:1086650050A77BFF7A62798A1257419013D9125825
:108675008A9015DE124D799013E812588A1258B176
:108685001259401250A71256E7129088129C5C7E30
:10869500637FAF7D0312885C7B017A1279D912570B
:0486A500E602940B4A
:1081C9009006D312581A7B019012871257399013CF
:1081D900A5F09006D712581A90128A12573990139F
:1081E900B8F09006DB12581A90128D125739901375
:1081F900CCF09006DF12581A90129012573990134A
:10820900CFF09006E312581A90129312573990132F
:10821900D1F0E4FD125858EF7802C333CE33CED8EB
:10822900F91259A4E07BFFB406067A6279E4800466
:108239007A6279E01258589012F11256D6124D7995
:058249000DEDB405CFAE
:01824E00220D
:109204001259177A4E793CF4700A743C65827004E2
:10921400744E658360161259177A6D797AF4700A60
:10922400747A65827004746D65837003129BEE22F8
:108D2E00E4901776F0901776E0FFC3648094995024
:108D3E0036EF3395E0FE74FB2FF58274133EF58308
:108D4E00E09017766009E025E02407A3F080031277
:108D5E0059957F0312928F901777E0FF1299DB904F
:078D6E001776E004F080BE5F
:018D750022DB
:10891B00E4901778F0901778E0FFC3648094995037
:10892B004B9013A4E075F07D900749124D44EF3343
:10893B0095E0FE75F005EF124D44EE75F005A4259C
:10894B0083F583E0540F9017786009E025E0240746
:10895B00A3F080031259957F0312928F901779E041
:0C896B00FF1299DB901778E004F080A95F
:0189770022DD
:0F93BB00E490177AF090177AE0FFC394195019D5
:1093CA00EF1259967F0A12928F90177BE0FF12993B
:0193DA00DBB7
:0893DB0090177AE004F080DD38
:0193E3002267
:104E3C009013A3E0600D7F0312928F7F381299DBE1
:104E4C0012891B901497E0FF1292E8500890123DC3
:104E5C00E0901497F0901497E0FF642C6004EFB48A
:104E6C00290890123DE0901497F0901497E0FF9071
:104E7C00123DF012572C75F005EFA4F58285F083E6
:104E8C0012493E540F901497600AE012578FC3E9F1
:104E9C00948A8008E01256F8C3E99471901707F0D1
:104EAC00901707E0125727E92F125865C4540F903A
:104EBC001708F0900001124AB5FF901709E5F0F0C1
:104ECC00A3EFF0900003124AB5FF90170BE5F0F03A
:104EDC00A312587F24FA1257CDC333CE33CED8F950
:104EEC001259C2E024FE600A14600C14600E2404F3
:104EFC0070161258138008125878800312592C908F
:104F0C0013DA1256D0124D7912579E9012EFF07B95
:104F1C00FF7A62799B125741125881FF9015DEE59A
:104F2C00F0F0A3EFF09013A3E07BFF60067A6279B8
:104F3C006780047A62796A9015E0124D797B017A68
:104F4C001279EF9015E3124D79ED1258C6124D59A6
:104F5C00124D8E9015E6124D797B017A1379A712BA
:104F6C0050A71257CEC333CE33CED8F924E0F582F6
:104F7C0074063EF583E07BFFB4051B7A6279AE12B2
:104F8C0057411257EC90170BE0FFA3E09015E0CFC0
:104F9C00F0A3EFF080127A6279BF1257411257ECEE
:104FAC007A6279D0A3124D791259401250A7125936
:104FBC0009400D1256E7129088E49014D7F0A3F034
:104FCC00129C5C7E637F327D0612885C7B017A12B8
:084FDC0079CD1257E602940B97
:069C68009012E8EFF0226B
:099BF700EF543FFFE4125839223B
:108DBC007E00EF7806C333CE33CED8F912582DD3BC
:108DCC0094C6EE9403400A9012CE7403F0A374C6BA
:108DDC00F09012E8E0FFE4D39F5019EFC3941950C0
:108DEC00139012CEE0FEA3E0FF9012E8125947EE6A
:048DFC00F0A3EFF001
:018E0000224F
:0C9B8D009012E8E024FB125844EFF02294
:0D9B5C00EF543FFF9012CEE4F0A3EFF02293
:109581007E00EF7806C333CE33CED8F912582DD3EF
:1095910094F4EE940140047E017FF4125747EEF0FB
:0395A100A3EFF045
:0195A40022A4
:0F9B07009012EAEFF0E0C3940540037404F022DB
:0F9B16009013D9EFF0E0C3940D4003740CF022CC
:0F9B25009013E8EFF0E0C3940D4003740CF022AE
:03000000024000BB
:03000300025003A5
:03000B000250069A
:030013000250098F
:03001B0002500C84
:0300230002500F79
:03002B000250126E
:0300330002501563
:03003B0002501858
:0300430002501B4D
:03004B0002501E42
:0300530002502137
:03005B000250242C
:0300630002502721
:03006B0002502A16
:0300730002502D0B
:03007B0002503000
:03008300025033F5
:03008B00025036EA
:03009300025039DF
:03009B0002503CD4
:0300A30002503FC9
:10400000787FE4F6D8FD9000007F007E20E4F0A3E6
:0A401000DFFCDEFA75816F024055F7
:10401A0002409AE493A3F8E493A34003F68001F2E2
:10402A0008DFF48029E493A3F85407240CC8C333A7
:10403A00C4540F4420C8834004F456800146F6DF76
:10404A00E4800B01020408102040809065F7E47EAA
:10405A00019360BCA3FF543F30E509541FFEE4936B
:10406A00A360010ECF54C025E060A840B8E493A332
:10407A00FAE493A3F8E493A3C8C582C8CAC583CA5D
:10408A00F0A3C8C582C8CAC583CADFE9DEE780BE15
:01676E00002A
:10482F00E709F608DFFA8046E709F208DFFA803E6B
:10483F0088828C83E709F0A3DFFA8032E309F60858
:10484F00DFFA8078E309F208DFFA807088828C83C0
:10485F00E309F0A3DFFA806489828A83E0A3F60874
:10486F00DFFA805889828A83E0A3F208DFFA804C4E
:10487F0080D280FA80C680D4806980F28033801025
:10488F0080A680EA809A80A880DA80E280CA80338E
:10489F0089828A83ECFAE493A3C8C582C8CCC58306
:1048AF00CCF0A3C8C582C8CCC583CCDFE9DEE780D6
:1048BF000D89828A83E493A3F608DFF9ECFAA9F055
:1048CF00EDFB2289828A83ECFAE0A3C8C582C8CCAB
:1048DF00C583CCF0A3C8C582C8CCC583CCDFEADEC4
:1048EF00E880DB89828A83E493A3F208DFF980CC26
:1048FF0088F0EF60010E4E60C388F0ED2402B4041F
:10490F000050B9F582EB2402B4040050AF232345C5
:06491F00822390487F7323
:10492500BB010689828A83E0225002E722BBFE0290
:09493500E32289828A83E49322C3
:10493E00BB010CE58229F582E5833AF583E022502E
:10494E0006E92582F8E622BBFE06E92582F8E22278
:0D495E00E58229F582E5833AF583E4932292
:10496B00BB010989828A83F8E028F022500327F7DC
:10497B0022BBFE05F8E328F3228A838982F8E493AD
:02498B002822E0
:10498D00BB010689828A83F0225002F722BBFE0109
:02499D00F32203
:10499F00F8BB010DE58229F582E5833AF583E8F04E
:1049AF00225006E92582C8F622BBFE05E92582C8FA
:0249BF00F222E2
:1049C100EF8DF0A4A8F0CF8CF0A428CE8DF0A42E0A
:0249D100FE22C4
:1049D300BC000BBE0029EF8DF084FFADF022E4CCC8
:1049E300F875F008EF2FFFEE33FEEC33FCEE9DEC91
:1049F300984005FCEE9DFE0FD5F0E9E4CEFD22EDD7
:104A0300F8F5F0EE8420D21CFEADF075F008EF2F20
:104A1300FFED33FD4007985006D5F0F222C398FD11
:054A23000FD5F0EA22AE
:104A2800C2D5EC30E709B2D5E4C39DFDE49CFCEEA9
:104A380030E715B2D5E4C39FFFE49EFE1249D3C305
:104A4800E49DFDE49CFC80031249D330D507C3E400
:064A58009FFFE49EFE2218
:104A5E00C5F0F8A3E028F0C5F0F8E58215827002E3
:064A6E001583E038F02280
:104A7400A3F8E0C5F025F0F0E582158270021583F5
:064A8400E0C838F0E82252
:104A8A00BB010A89828A83E0F5F0A3E022500687F7
:104A9A00F009E71922BBFE07E3F5F009E3192289B9
:0B4AAA00828A83E493F5F074019322EC
:104AB500BB0110E58229F582E5833AF583E0F5F03F
:104AC500A3E0225009E92582F886F008E622BBFE1C
:104AD5000AE92582F8E2F5F008E222E5832AF58362
:084AE500E993F5F0A3E9932227
:104AED00BB010DC58229C582C5833AC583024A5EC5
:104AFD005011C58229F808E5F026F618F5F0E58283
:104B0D0036F622BBFE11C58229F808E225F0F5F034
:104B1D00F218E23582F222F8E58229F582E5832A40
:0D4B2D00F58374019325F0F5F0E493382230
:104B3A00F8BB0111E58229F582E5833AF583E8F0AD
:104B4A00E5F0A3F0225009E92582C8F608A6F0226A
:0D4B5A00BBFE09E92582C8F2E5F008F22251
:0D4B6700EF2BFFEE3AFEED39FDEC38FC229D
:104B7400E88FF0A4CC8BF0A42CFCE98EF0A42CFCE0
:104B84008AF0EDA42CFCEA8EF0A4CDA8F08BF0A45E
:104B94002DCC3825F0FDE98FF0A42CCD35F0FCEBBD
:104BA4008EF0A4FEA9F0EB8FF0A4CFC5F02ECD3982
:0F4BB400FEE43CFCEAA42DCE35F0FDE43CFC22EF
:104BC30075F008758200EF2FFFEE33FECD33CDCCA9
:104BD30033CCC58233C5829BED9AEC99E58298402C
:104BE3000CF582EE9BFEED9AFDEC99FC0FD5F0D609
:104BF300E4CEFBE4CDFAE4CCF9A88222B800C1B933
:104C03000059BA002DEC8BF084CFCECDFCE5F0CB70
:104C1300F97818EF2FFFEE33FEED33FDEC33FCEBA9
:104C230033FB10D703994004EB99FB0FD8E5E4F964
:104C3300FA227818EF2FFFEE33FEED33FDEC33FC51
:104C4300C933C910D7059BE99A4007EC9BFCE99A45
:104C5300F90FD8E0E4C9FAE4CCFB2275F010EF2F8A
:104C6300FFEE33FEED33FDCC33CCC833C810D7078A
:104C73009BEC9AE899400AED9BFDEC9AFCE899F8C5
:0E4C83000FD5F0DAE4CDFBE4CCFAE4C8F92258
:108ECD00C2D5E830E70FB2D5E4C39BFBE49AFAE4D0
:108EDD0099F9E498F8EC30E717B2D5128F03124BDD
:108EED00FFE4C39BFBE49AFAE499F9E498F8800354
:108EFD00124BFF30D50DE4C39FFFE49EFEE49DFDB4
:048F0D00E49CFC22C2
:104C9100EB9FF5F0EA9E42F0E99D42F0EC6480C89A
:064CA10064809845F0223A
:104CA700EB9FF5F0EA9E42F0E99D42F0E89C45F063
:014CB70022DA
:104CB800E8600FECC313FCED13FDEE13FEEF13FFDA
:034CC800D8F122FE
:104CCB00E8600FEFC333FFEE33FEED33FDEC33FC47
:034CDB00D8F122EB
:0C4CDE00E0FCA3E0FDA3E0FEA3E0FF2249
:0C4CEA00E0F8A3E0F9A3E0FAA3E0FB224D
:0C4CF600ECF0A3EDF0A3EEF0A3EFF02231
:104D0200A8828583F0D083D082124D19124D1912D8
:104D12004D19124D19E473E493A3C583C5F0C583FD
:104D2200C8C582C8F0A3C583C5F0C583C8C582C8FB
:014D3200225E
:104D3300F5F0C582A4C582C5F0C583A42583F58398
:014D4300224D
:0C4D4400A42582F582E5F03583F583227A
:094D5000E6FB08E6FA08E6F92288
:094D5900E0FBA3E0FAA3E0F9225B
:104D6200F8E0FBA3A3E0F925F0F0E58215827002DA
:074D72001583E0FA38F0227E
:094D7900EBF0A3EAF0A3E9F0223B
:0C4D8200E493FB740193FA740293F9228D
:104D8E00BB010789828A83024D595005E9F8024D0D
:104D9E0050BBFE05E9F8024E3389828A83024D82AA
:104DAE00D083D082F8E4937012740193700DA3A394
:104DBE0093F8740193F5828883E4737402936860A8
:064DCE00EFA3A3A380DFA8
:064DD4008A838982E4736A
:104DDA00EC8EF0A4CCC5F0CCCDF8EFA4CEC5F02D66
:104DEA00FDE43CFCE8A42EC8C5F03DFDE43CFCEF24
:0D4DFA00A4FFE5F028FEE43DFDE43CFC22B2
:10504200E51724DBF582E43415F583E00517229099
:1050520015D83010039015DBE475F001124D620291
:1050620049252009E97F2ED2098018EF540F249098
:10507200D43440D4FF300D0BEF24BFB41A005003D8
:105082002461FFE51860021518051BE51B70020577
:105092001A30100E9015D8E475F001124D62EF022D
:1050A200498D0294327403D2108003E4C210F517C2
:1050B2009015D8124D79E4F518F51AF51BE518602C
:1050C200077F2012508580F57519FFC20AC209C2F6
:1050D2000BC20CC20EC20FC211125051FF700D3022
:1050E20010057F00125096AF1BAE1A22B4255FC284
:1050F200D5C20D125051FF24D0B40A00501A75F0D7
:105102000A781830D50508B6FF0106C6A426F6208F
:10511200D5047002D20C80D924CFB41A00EF500407
:10512200C2E5D20D025297D20A80C6D20980C0D2FD
:105132000B80BCD2D580BAD20E80B47F20125085AB
:10514200200B077401B5180040F1125042FF1250B3
:10515200850250BFD211D20F8095125042FB1250DD
:1051620042FA125042F94A4B700679687A537BFF31
:10517200200B2EE518602A7E008E8275830012496C
:105182003E60060EEE651970F0C2D5EBC0E0EAC0D3
:10519200E0E9C0E0EE1252DED0E0F9D0E0FAD0E071
:1051A200FB124925FF60AAEBC0E0EAC0E0E9C0E0DB
:1051B200125085D0E02401F9D0E03400FAD0E0FBAF
:1051C200E5190460DCD519D980877BFF7A5279DA38
:1051D200D20B809C791080027908C20FC21180081C
:1051E200D2D5790A8004790AC2D5E519047002F58C
:1051F20019E4FAFDFEFF125042FC7B08200A13124A
:105202005042FD7B1030090A125042FE125042FFFA
:105212007B20EC3382D592D55013C3E43009069F2C
:10522200FFE49EFEE4200A039DFDE49CFCE4CBF82F
:10523200C20AEC700CCFCECDCCE824F8F870F38023
:1052420017C3EF33FFEE33FEED33FDEC33FCEB33EC
:10525200FB994002FB0FD8E9EB300A05F8D0E0C415
:1052620048B20AC0E00AEC4D4E4F78207B0070C273
:10527200EAB5190040BCC0E01252E0D0F0D0E02004
:105282000A04C4C0E0C4B20AC0F012506ED0F0D515
:10529200F0EB0250BF124DAE515C5351D658512D16
:1052A2004C51294251DA4F51E24451E249514243B1
:0852B20051E85551CC4651CCE6
:1052BA004551CC4753885051312D51352E51582BD9
:1052CA0051392351562053712A50F1480000515048
:1052DA003F3F3F00790AA2D5200C14300E09B910BD
:1052EA00020404B9080104A2D5200F0250010420C7
:1052FA000B68920BB518005034C0E07F20300C19AF
:10530A007F30A20B720F720E500F125337C20BC2AC
:10531A000FC20EC2117F30800F300E03E9C0E012B7
:10532A005085300E03D0E0F9D0E0B518CC300E1716
:10533A007F30B9100C1250857F58300D077F788066
:10534A0003B90803125085300B057F2D0250857F63
:10535A00202011F87F2B200FF322920B80CF286E8A
:10536A00756C6C2900D20A125042300AF8C20A78C7
:10537A001830D50108F60250F12D50434958125001
:10538A00422403B405004001E490538393125076FB
:0D539A00743A125076D20C7518040251D6E8
:0C9B9900EE30E707C3E49FFFE49EFE22CD
:104E0700EF4E6012EF60010EEDBB010B89828A83C2
:104E1700F0A3DFFCDEFA2289F05007F709DFFCA9CF
:0C4E2700F022BBFEFCF309DFFCA9F02226
:094E3300E2FB08E2FA08E2F922B0
:10943200EFB40A07740D12943D740A309811A8997A
:10944200B8130CC2983098FDA899C298B811F6309A
:0794520099FDC299F5992272
:00000001FF
